:10000000E7280530AA00A530AB00AB0B0528AA0BEA
:10001000032800348600003066000515851005149D
:100020000510FF3066000511851405140608AF00A1
:10003000AF1705100514861F1F2805101A28051074
:100040003228860000306600051185100514051061
:10005000FF30660085140514861F302805102B28F4
:10006000051000342F1C0034AF1C00342F1D003449
:10007000AF1D00343930AF07AF172F082128831385
:1000800010088D0203184B2801308E0203184B28EC
:100090008F02031C831711088E02031853280130A6
:1000A0008F02031C831712088F02031C831700346E
:1000B00010088D07031C5F288E0F5F288F0A110818
:1000C0008E0703188F0A12088F0700340730AA0022
:1000D000193084002F308000840AAA0B6B280F305F
:1000E000920042309100403090003F20990A3A300F
:1000F00019060319662A831F7528582001309200BB
:1001000086309100A03090003F209A0A831F8428F7
:100110005820920127309100103090003F209B0A18
:10012000831F8E28582003309100E83090003F2034
:100130009C0A831F972858209101643090003F202B
:100140009D0A831F9F2858200A3090003F209E0A56
:10015000831FA62858200D089F079F0A00343730B8
:10016000620010306500851105118F018101960133
:10017000051505110C08AA008515FA30AB00C62834
:1001800000000000000000000000000001089602CE
:10019000031DCC280000CE2803188F0A960000000B
:1001A00000000000AB0BC028AA0BBD288511010878
:1001B0008E009602031CDE28031D8F0A8D018D031D
:1001C0000515051101080E060319DF280034850105
:1001D00010306500860100306600012001200120FA
:1001E0003830860005140120051005140120051083
:1001F000051401200510061221200C3021200130A9
:1002000021200630212020300A2020300A202030F2
:100210000A2043300A202E300A2054300A20413070
:100220000A2056300A2045300A2052300A204E302B
:100230000A2049300A2045300A2052300A20063070
:10024000AC00C830AD000120AD0B2329AC0B212937
:10025000013021200630212020300A2020300A20C1
:1002600045300A204C300A2045300A2043300A200D
:1002700054300A2052300A204F300A204E300A20D3
:1002800049300A2051300A2055300A2045300A20D2
:100290000630AC00C830AD000120AD0B4C29AC0BD2
:1002A0004A29013021200630212020300A20203028
:1002B0000A2020300A2020300A2050300A205230F4
:1002C0000A2041300A2054300A2049300A20513097
:1002D0000A2055300A2045300A2020300A202030DC
:1002E0000A200630AC00C830AD000120AD0B7529E6
:1002F000AC0B7329013021200630212014308C00F2
:10030000AF20662030301906031D8A2930301A06C6
:100310000319C929823021200230AA001930840033
:1003200030300006031D9A2920300A20840AAA0BC7
:1003300090299F2900080A20840AAA0B9A292E30A6
:100340000A200530AA0000080A20840AAA0BA32963
:1003500020300A204D300A2048300A207A300A2006
:1003600020300A2020300A207E2914308C00AF2053
:10037000662030301906031D8A2932301A0203180C
:100380008A2930301A06031DC92930301B0603198B
:10039000F229823021200530AA0019308400303043
:1003A0000006031DD92920300A20840AAA0BCF2970
:1003B000DE2900080A20840AAA0BD9292E300A2037
:1003C00000080A20840A00080A2020300A206B3026
:1003D0000A2048300A207A300A2020300A202030B3
:1003E0000A20B529C8308C00AF20662030301906AD
:1003F000031DB52932301A020318B52930301A0608
:10040000031D062A30301B060319422A82302120A0
:100410000430AA001930840030300006031D162A6B
:1004200020300A20840AAA0B0C2A1B2A00080A2062
:10043000840AAA0B162A2E300A2000080A20840AF1
:1004400000080A20840A00080A2020300A206B30A5
:100450000A2048300A207A300A2020300A20203032
:100460000A20F229C8308C00AF20662030301906EF
:10047000031D062A30301A06031D062A32301B02DD
:100480000318062A823021200730AA001930840080
:1004900030300006031D522A20300A20840AAA0B9D
:1004A000482A572A00080A20840AAA0B522A203018
:1004B0000A2048300A207A300A2020300A202030D2
:1004C0000A2020300A2020300A20322A0130212040
:1004D0008430212044300A2045300A2042300A204E
:1004E0004F300A2052300A2044300A2045300A207A
:1004F0004D300A2045300A204E300A2054300A2060
:06050000023021207E29DB
:00000001FF
